:020000040000FA
:02000000A02836
:080008008D00030E8E00640060
:100010008C0A0C08F03A031917200C08783A0319D7
:1000200085150E0E83008D0E0D0E0B110900851126
:100030008C018F0A990A900A10083C3A031D0800A7
:100040009001910A08008207C034D034D834DC34DF
:10005000DE34DF34CF34C734C334C134FA34E73448
:10006000E534F334FD34ED34FF34FF34FF34FF3432
:10007000FF34FF34FF34FF34FF34FF34D234EA342A
:10008000E134CA34C934BA340034D934AD34FF341D
:10009000FF34FF34FF34A134C9349234FF34D534F3
:1000A0008C34FF34AA34CD34C034D034D834DC346A
:1000B000DE34DF34CF34C734C334C1348734FF3443
:1000C000FF34CE34FF34B334FF34FA34E734E5344C
:1000D000F334FD34ED34F134EF34FB34E834F234EE
:1000E000EB34F834F934F034E934E234F534F734ED
:1000F000FC34F634EE34F434E634E434E33482078A
:100100000D34083404340F340234003406340B3414
:100110000134093405340A3403340E3407340C3402
:10012000820705340A3414341E34283432343C3403
:100130007834F034013401340134013401340134B1
:100140000B118B178B1681016400C330831681005D
:100150008312810183168501BF30860083128510CA
:10016000051406171A30562394001B3056239A00A4
:100170001C3056239B001D30562392001E30562300
:100180009D001F3056239E008510861EC428861FA2
:10019000F028061ACE28861EC428C7280608061A84
:1001A000CF280F397F2097000E3A0319FD28C72862
:1001B00006080F397F20003A031DFD28861ADE2825
:1001C000051085142F23203097002F238312170842
:1001D0005623E822970A17083B3A031DE6280F2901
:1001E0009C0103012B2303012B239C0A861BC4289B
:1001F0001C08A03A0319FD28F128061AD828861AE7
:10020000FD280229051085142F2397018312170852
:100210005623E822970A1708083A031D06293D309D
:100220005623880A5C230808003A031D1B293C302A
:100230005623880A5C232F23372398018C018F01D2
:1002400090019101861A29290F081D060319C42857
:1002500022298C018F01861A32290F081D060319E5
:100260009E2A2B29980A1808103A03199803851416
:100270008C0199010514140819060319CC2A061AD1
:100280006C29861A3A2978308C008F01861E4929FC
:100290003A290F08013A031D46291A081102031CC6
:1002A0006029051008309700831217085623E822AA
:1002B000970A1708103A031D54292F239001910122
:1002C00037232929861E6029061E622906080F3950
:1002D0007F20061A6929080006080F397F20970039
:1002E0000F3A03197C2917080E3A03197C291708BD
:1002F0000A3A03198A293A29061A7C29861E602996
:10030000061E7E2906080F397F209700093A031937
:10031000112A3A29061A8A2905106221083A031D72
:100320003A296221093A031D3A296221073A031D3D
:100330003A29861A992905102F235330E82245308F
:10034000E8225430E8222F2337238F010F080A3A7E
:1003500003193A29061EA62906080F397F20061A16
:10036000AF29861AB12997000E3A03193A291708BE
:100370000F3A03191C2A17080A3A0319F529170816
:100380000B3A0319EB291708093A0319012A05103A
:1003900017082F231708E8222F235230E8222F2393
:1003A0000514851090209700900191010C08103AD7
:1003B0000319851517081106031DD6290510851484
:1003C0002F235130E8225230E8225630E8222F23E2
:1003D00085100514C428061705102F234F30E82276
:1003E0004E30E8222F2305149929061305102F23D8
:1003F0004F30E8224630E8224630E8222F23051409
:10040000992905102F235130E8225230E822543028
:10041000E8222F2305140C08103A031985158510BE
:100420000B2A861A112A05102F234330E8224C305C
:10043000E8222F230514C42805101A3092004F30EB
:10044000E8225030E8224E30E8222030E8229C0199
:100450003C3056239F0093221F089B223D30562399
:100460009F0093221F089B222030E8229C0A1C0830
:10047000023A031D282A2030E8223D30E8222030AD
:100480005130E8225330E8224F30E8222030E82271
:100490009C013E3056239F0093221F089B223F3031
:1004A00056239F0093221F089B222030E8229C0A9B
:1004B0001C08023A031D492A2030E8224B30E8226A
:1004C00005141D30562392008F018C010F080A3A43
:1004D00003199929061E662A06080F397F20061A75
:1004E0006F2A861A712A97000E3A0319992917085C
:1004F0000F3A031D99293C308900880189005C234B
:100500003D30890088015C233E30890088015C23EE
:100510003F30890088015C2305102F235230E822E8
:100520002F23051499299700970C970C970C170CFB
:100530000F39E82208000F39E822080085108C01E5
:100540008F01861A32290F081E060319A82AA12A2C
:100550001808970005309702031CC428851405105D
:100560002F2310309700831217085623E822970A8A
:100570001708183A031DB32A2F23851005143F309E
:100580005623880A5C230808003A031DCB2A3E3014
:100590005623880A5C23C42818305623E8221930D1
:1005A0005623E8222F238510861AD42A78308C000F
:1005B0008F01861AD42A0F08013A031DD92A8514FF
:1005C00005102F233723051037232F2385109E2A4C
:1005D00023209300FF3A031908001308003A031977
:1005E000232B07309600930D031CF82A960BF32A51
:1005F000930D031C022305231423960BF82A1423BE
:10060000142308000523052308001208950005158A
:1006100003012B231B082B23051103012B231B088C
:100620002B23950B072B08001208950005110301D9
:100630002B231B082B23051103012B231B082B2322
:10064000950B162B080014231423142314231423AE
:10065000142314230800013E031D2B2B08007830BF
:100660008C008F010F08013A031D322B0800051082
:1006700016309500051503012B23FF302B230511A0
:1006800003012B23FF302B23950B3A2B16309500BB
:10069000051503012B237F302B23051103012B2389
:1006A0007F302B23950B482B0514080089008316F7
:1006B000081483120808080083168B130815553098
:1006C0008900AA30890088148818642B0811081240
:0606D0008B1783120800E5
:1007D0005600650072002E0031002E0031006900C5
:1007E000320036002D00300037002D00300032007E
:1007F0002A004F0048003300480052004B002A00F6
:02400E00FD3F74
:104200004F00480033005200410043002D002D00B4
:104210004F00480033005200410043002D002D00A4
:104220004F00480033005200410043002D002D0094
:1042300043004C003C000A00EF001100080007009A
:104240004400450020004F00480033005200410068
:10425000430020004C004100480054004900200069
:104260004B00500032003000540058002D002D004B
:104270002D002D002D002D0000000000000000008A
:00000001FF
